:0200000480007A
:100000009705000093854506130540006B10B50069
:10001000EF004005130510006B0005001385C108B3
:100020001386810C3306A64093050000EF10403C78
:1000300017150000130505AFEF00502AEF005034EC
:08004000EF00D0156F00D02A7B
:10004800B70700009387070063880700371500800B
:10005800130505B26F0010286780000013054000E3
:100068006B000500972100009381C179F3261002E7
:100078009396A601732600029315A6001316260070
:1000880037F1FF6F3301B1403301D1403301C10073
:10009800F326100263860600130500006B000500B6
:1000A80067800000D772850007E0051233055540C8
:1000B80093922200B38555008760061233065600D6
:1000C8005781000227E10602B3865600E31E05FCAD
:1000D800D72021B667800000130101FD2326810285
:1000E80013040103232EA4FC232CB4FC232AC4FCF0
:1000F8008327C4FD83A707002326F4FE930744FD46
:100108002322F4FE832744FE03C707008327C4FE87
:100118002380E7008327C4FE93871700032744FE44
:10012800034717002380E7008327C4FE938727002F
:10013800032744FE034727002380E7008327C4FEE4
:1001480093873700032744FE034737002380E700DF
:100158008327C4FE938747002326F4FE232404FE46
:100168006F004003832784FE032784FDB307F7004D
:1001780003C707008327C4FE2380E7008327C4FE44
:10018800938717002326F4FE832784FE938717009E
:100198002324F4FE832744FD032784FEE344F7FC6D
:1001A8008327C4FE2320F4FE832704FE93F7370039
:1001B800032704FEB307F7002320F4FE832704FE79
:1001C8002326F4FE8327C4FD0327C4FE23A0E700EB
:1001D800130000000324C10213010103678000001B
:1001E800130101FC232E8102130401042326A4FC1D
:1001F8002324B4FC8327C4FC83A707002326F4FE2A
:100208009307C4FD2322F4FE8327C4FE03C7070017
:10021800832744FE2380E700832744FE9387170043
:100228000327C4FE034717002380E700832744FE03
:10023800938727000327C4FE034727002380E7008E
:10024800832744FE938737000327C4FE03473700FC
:100258002380E7008327C4FE938747002326F4FE04
:10026800232404FE6F004003832784FE032784FCB5
:10027800B307F7000327C4FE034707002380E700FE
:100288008327C4FE938717002326F4FE832784FE62
:10029800938717002324F4FE8327C4FD032784FED5
:1002A800E344F7FC8327C4FE2320F4FE832704FEDF
:1002B80093F73700032704FEB307F7002320F4FE63
:1002C800832704FE2326F4FE8327C4FC0327C4FEE9
:1002D80023A0E700130000000324C1031301010455
:1002E80067800000130101FF232681001304010128
:1002F800130000000324C1001301010167800000FE
:10030800130101FE232E8100130401022326A4FEFB
:100318002324B4FE832784FE3727000023A2E700A6
:1003280093070000138507000324C101130101028C
:1003380067800000130101FE232E1100232C810089
:10034800130401022326A4FEB7270080138507B3F0
:10035800EF00C04F93071000138507008320C101E9
:10036800032481011301010267800000130101FDCC
:10037800232611022324810213040103232EA4FC43
:10038800232CB4FC232AC4FCB70700712326F4FEEF
:10039800B70700722324F4FE930730002322F4FEEB
:1003A800130744FE9307C4FE130640009305070095
:1003B80013850700EFF05FD21307C4FD9307C4FE4F
:1003C800130640009305070013850700EFF0DFD000
:1003D800130784FD9307C4FE130640009305070026
:1003E80013850700EFF05FCF130744FD9307C4FEA2
:1003F800130640009305070013850700EFF0DFCDD3
:1004080083A74107E7800700130704FE930784FECC
:100418009305070013850700EFF09FDC832704FE90
:10042800138507008320C1020324810213010103FD
:1004380067800000130101FD232611022324810295
:1004480013040103232EA4FC232CB4FC232AC4FC8C
:10045800B70700712324F4FEB70700722326F4FEC1
:10046800930740002322F4FE130744FE930784FEFB
:10047800130640009305070013850700EFF0DFC55A
:100488001307C4FD930784FE130640009305070075
:1004980013850700EFF05FC4130784FD930784FEFC
:1004A800130640009305070013850700EFF0DFC22D
:1004B800130744FD930784FE1306400093050700C5
:1004C80013850700EFF05FC183A74107E7800700A6
:1004D800832744FD138507008320C102032481027A
:1004E8001301010367800000130101FD2326110297
:1004F8002324810213040103232EA4FC232CB4FC1F
:10050800232AC4FCB70700712326F4FE9307500082
:100518002324F4FE130784FE9307C4FE1306400049
:100528009305070013850700EFF01FBB1307C4FDF1
:100538009307C4FE130640009305070013850700C0
:10054800EFF09FB99307C4FE032644FD832584FD7D
:1005580013850700EFF05FB883A74107E78007001E
:10056800832744FD138507008320C10203248102E9
:100578001301010367800000130101FD2326810296
:1005880013040103232EA4FC8327C4FD63D80700AA
:100598008327C4FDB307F040232EF4FC0327C4FDD2
:1005A800B73700009387078063D8E700B7370000A4
:1005B80093870780232EF4FC83A781072326F4FE64
:1005C80003A781078327C4FD3307F70023ACE1069F
:1005D8008327C4FE138507000324C1021301010306
:1005E80067800000130101FE232E1100232C8100D7
:1005F800130401022326A4FE13050000EF00001EC9
:10060800130000008320C1010324810113010102AA
:1006180067800000130101FD2326110223248102B3
:1006280013040103232EA4FC232CB4FC232AC4FCAA
:10063800B70700712326F4FEB70700722324F4FEDF
:10064800930770002322F4FE130744FE9307C4FEA9
:10065800130640009305070013850700EFF0DFA796
:100668001307C4FD9307C4FE130640009305070053
:1006780013850700EFF05FA6130784FD9307C4FEF8
:10068800130640009305070013850700EFF0DFA469
:10069800130744FD9307C4FE1306400093050700A3
:1006A80013850700EFF05FA383A74107E7800700E2
:1006B800130704FE930784FE9305070013850700BC
:1006C800EFF01FB2832704FE138507008320C102C1
:1006D800032481021301010367800000130101FF55
:1006E800232611002324810013040101B727008069
:1006F800138547B4EF008015130000008320C10064
:10070800032481001301010167800000130101FF28
:10071800232611002324810013040101EF00800E19
:1007280093070500138507008320C1000324810077
:100738001301010167800000130101FF2326110046
:100748002324810013040101B7270080138587B68D
:10075800EF00C00F130000008320C10003248100B4
:100768001301010167800000130101FF2326110016
:100778002324810013040101B72700801385C7B81B
:10078800EF00C00C83A781099386170023ACD1081A
:10079800138507008320C100032481001301010190
:1007A80067800000130101FF232611002324810024
:1007B80013040101B7270080138587BBEF000009E8
:1007C800130000008320C1000324810013010101EC
:1007D800678000006B10B500678000006B000500A3
:1007E800678000006B40B500678000006B20050043
:1007F800678000006B3000006780000073251002DE
:100808006780000073250002678000001305400020
:100818006B000500F32610029396F600732600027B
:100828009315A6001316260037F1FF6F3301B14068
:100838003301D1403301C100F3261002638606005C
:10084800130500006B00050067800000130141FFDD
:10085800232011002322B100834505006388050089
:10086800EF00C001130515006FF01FFF8320010082
:10087800832541001301C10067800000B702010011
:1008880023A0B20067800000130101FD2326110296
:100898002324810213040103232EA4FC0327C4FD8F
:1008A8009307F00063E4E702B72700800327C4FD3D
:1008B8001317270093878700B307F70083A707005C
:1008C80013850700EFF09FF86F00400793070002B9
:1008D8002326F4FEA30504FE8327C4FE9387C7FFDF
:1008E8000327C4FDB357F70093F7F7002322F4FE5C
:1008F800832744FE6386070093071000A305F4FED0
:100908008347B4FE63820702B7270080032744FEAB
:100918001317270093878700B307F70083A70700FB
:1009280013850700EFF09FF28327C4FE9387C7FF64
:100938002326F4FE8327C4FEE340F0FA8320C10295
:10094800032481021301010367800000130101FEE3
:10095800232E1100232C8100130401022326A4FE58
:100968002324B4FE0325C4FEEFF05FEE032584FEC6
:10097800EFF09FF1B72700801385C7C1EFF01FED97
:10098800130000008320C101032481011301010227
:1009980067800000130101FD232611022324810230
:1009A8001304010313051000EFF05FE3930700023F
:1009B8002322F4FE832744FE93972700138507001C
:1009C800EF004025930705002320F4FE832744FE0B
:1009D8009397270013850700EF00C02393070500AE
:1009E800232EF4FC832744FE9397270013850700E2
:1009F800EF00402293070500232CF4FC232604FE75
:100A08006F0080058327C4FE93972700032704FE01
:100A1800B307F7001307100023A0E7008327C4FEDD
:100A2800939727000327C4FDB307F70013071000A7
:100A380023A0E7008327C4FE93972700032784FD9C
:100A4800B307F7001307100023A0E7008327C4FEAD
:100A5800938717002326F4FE0327C4FE832744FE4A
:100A6800E342F7FA832684FD0326C4FD832504FEAA
:100A7800032544FEEFF00FE3232404FE6F00C002B9
:100A8800832784FE93972700032784FDB307F70085
:100A980083A7070013850700EFF01FDF832784FE75
:100AA800938717002324F4FE032784FE832744FE3C
:100AB800E348F7FC13050000EFF05FD213000000D5
:100AC800138507008320C102032481021301010357
:100AD80067800000930505009306000013060000D8
:100AE800130500006F005024130101FF9305000057
:100AF800232481002326110013040500EF00502C45
:100B080003A501078327C50363840700E78007005F
:100B180013050400EFF01FAD130101FF232481002A
:100B28002322910037240080B72400809387440053
:100B3800130444003304F4402326110013542440C2
:100B480063020402931424009384C4FFB384F40062
:100B580083A704001304F4FF9384C4FFE78007000D
:100B6800E31804FE8320C10003248100832441008C
:100B78001301010167800000130101FF2324810094
:100B8800232021013724008037290080930704009F
:100B9800130909003309F940232611002322910083
:100BA8001359294063000902130404009304000048
:100BB800832704009384140013044400E78007008B
:100BC800E31899FE37240080372900809307040032
:100BD800130949003309F9401359294063000902F0
:100BE8001304040093040000832704009384140072
:100BF80013044400E7800700E31899FE8320C1002E
:100C08000324810083244100032901001301010109
:100C1800678000009305050003A501086F00000127
:100C28009305050003A501086F00103D130101FDA0
:100C380023229102232E310123261102232481022B
:100C480023202103232C4101232A51012328610158
:100C58002326710123248101232291019384B50065
:100C6800930760019309050063E497069307000161
:100C780063ECB720EF00100593040001930780018F
:100C880013062000138981C6B307F90003A447009F
:100C9800138787FF6302E424832744008326C40064
:100CA8000326840093F7C7FFB307F40003A74700A0
:100CB8002326D60023A4C60013671700138509004E
:100CC80023A2E700EF005000130584006F00801C8A
:100CD80093F484FF63CA041A63E8B41AEF00807EB1
:100CE8009307701F63F8974693D79400638E071C89
:100CF80013074000636CF73E93D76400138697038D
:100D08001385870393163600138981C6B306D90065
:100D180003A44600938686FF638C860283274400DB
:100D28009305F00093F7C7FF3387974063C0E50248
:100D3800635807340324C400638C86008327440067
:100D480093F7C7FF33879740E3D4E5FE1306050002
:100D58000324090113088900630C0419832544003E
:100D68001307F00093F5C5FFB3879540634AF74032
:100D7800232A09012328090163D4073E9307F01F9A
:100D880063E6B73093D535009387150093973700FE
:100D980003254900B307F90083A6070093D525402A
:100DA800130710003317B7003367A700938587FF31
:100DB8002326B4002324D4002322E90023A087009B
:100DC80023A686009357264093061000B396F60094
:100DD800636AD712B3F7E600639407029396160086
:100DE8001376C6FFB3F7E60013064600639A0700BA
:100DF80093961600B3F7E60013064600E38A07FE4B
:100E08001305F00093183600B308190193850800FC
:100E18001303060003A4C500639A85006F00402FE2
:100E2800635207300324C4006384852E832744005B
:100E380093F7C7FF33879740E354E5FE8326C40042
:100E48000326840093E514002322B4002326D60049
:100E580023A4C600B3049400232A990023289900E8
:100E68009366170023A6040123A4040123A2D40037
:100E7800B307F4001385090023A0E700EF00C0645E
:100E8800130584006F0000019307C00023A0F90038
:100E9800130500008320C102032481028324410238
:100EA800032901028329C101032A8101832A4101FF
:100EB800032B0101832BC100032C8100832C4100EB
:100EC8001301010367800000930600201306000445
:100ED8001305F0036FF05FE303A4C70013062600B1
:100EE800E39C87DA0324090113088900E31804E75F
:100EF800032749009357264093061000B396F6003F
:100F0800E37AD7EC03248900832A440013FCCAFF40
:100F180063689C00B3079C401307F000634EF71208
:100F280083AA410903A741089307F0FF330A840104
:100F3800B38A54016308F732B71700009387F700A4
:100F4800B38AFA00B7F7FFFFB3FAFA0093850A00ED
:100F580013850900EF0080579307F0FF130B050076
:100F6800630AF52663664527938BC10983A70B009F
:100F7800B387FA0023A0FB00138707006306AA388B
:100F880083A641089307F0FF638EF638330A4B4176
:100F98003307EA0023A0EB00937C7B0063860C2ECA
:100FA800330B9B41B7170000130B8B00138AF7FF15
:100FB800B30A5B019387870033F74A01B3879741E8
:100FC800B387E74033FA470193050A001385090000
:100FD800EF00C04F9307F0FF6300F53A3305654112
:100FE800B30A450183A70B002324690193EA1A0079
:100FF800B307FA0023A0FB0023225B016308243314
:101008001306F000637886338326440013074CFFE9
:10101800137787FF93F61600B3E6E6002322D40081
:1010280093055000B306E40023A2B60023A4B6003B
:10103800636EE634832A4B0013040B0083A6010970
:1010480063F4F60023A8F10883A6C10863F8F6182C
:1010580023A6F1086F00801813E714002322E40088
:10106800B30494002324990093E71700138509001B
:1010780023A2F400EF004045130584006FF09FE1C0
:101088008326C400032684006FF01FC293D79500FF
:10109800130740006374F712130740016360F722D7
:1010A8009386C7051387B70593963600B306D9000C
:1010B80083A70600938686FF638AF61A03A747006C
:1010C8001377C7FF63F6E50083A78700E398F6FE6A
:1010D80083A6C700032749002326D4002324F4004D
:1010E80023A4860023A687006FF0DFCD13074001F5
:1010F8006378F710130740056360F71E93D7C400A1
:101108001386F7061385E706931636006FF0DFBFE0
:10111800130313009377330093858500E39C07CE70
:101128006F00C00FB307F40003A747008326C4006D
:10113800032684001367170023A2E7002326D6009E
:101148001385090023A4C600EF00003813058400A6
:101158006FF05FD413D63400938784006FF09FB28A
:10116800B305B40083A745001385090093E717006A
:1011780023A2F500EF004035130584006FF09FD1DE
:1011880013E714002322E400B3049400232A9900EF
:101198002328990013E7170023A6040123A40401B8
:1011A80023A2E400B305B4001385090023A0F500C9
:1011B800EF008031130584006FF0DFCD93D7650011
:1011C8009386970313878703939636006FF01FEE75
:1011D8006302241303248900832A440093FACAFF74
:1011E800B3879A4063E69A001307F000E346F7E6F0
:1011F80013850900EF00402D130500006FF09FC90B
:101208001386C7051385B705931636006FF0DFAF51
:1012180083A788001306F6FF6394171D937736009B
:10122800938888FFE39607FE0327490093C7F6FFD4
:10123800B3F7E7002322F90093961600E3E4D7CC2E
:10124800E38206CC33F7F600631A0700939616007C
:1012580033F7F60013034300E30A07FE13060300FF
:101268006FF05FBA938A0A016FF05FCE03254900D9
:1012780093552740130710003317B7003367A700AB
:101288002322E9006FF05FE5B71700001387F7FF27
:10129800330A5B01337AEA00B387474133FAE70040
:1012A80093050A0013850900EF0040229307F0FF19
:1012B800E316F5D2130A00006FF0DFD213074005DA
:1012C8006360F70893D7C5009386F7061387E70688
:1012D800939636006FF09FDD130740156360F7089B
:1012E80093D7F4001386870713857707931636007C
:1012F8006FF09FA1938BC10903A70B003387EA0006
:1013080023A0EB006FF0DFC793164A01E39A06C6E5
:1013180003248900B30A5C0193EA1A0023225401CA
:101328006FF0DFD123A261096FF01FC713040B0010
:101338006FF0DFD0930710002322FB006FF05FEB04
:10134800130740156362F70693D7F500938687075E
:1013580013877707939636006FF05FD513074055CC
:101368006362F70693D724011386D7071385C70747
:10137800931636006FF05F99938C8CFFB38A9A01AD
:10138800B38A6A41130A00006FF0DFC59305840031
:1013980013850900EF0040460324890083A70B004A
:1013A800832A44006FF09FC9130740556364F7020E
:1013B80093D725019386D7071387C70793963600D7
:1013C8006FF0DFCE9306803F1306F0071305E007A2
:1013D8006FF09F939306803F1307E0076FF01FCDD0
:1013E800832749006FF05FE51303F000130705003A
:1013F800637EC3029377F7006390070A6392050838
:10140800937606FF1376F600B386E6002320B7002E
:101418002322B7002324B7002326B70013070701A8
:10142800E366D7FE6314060067800000B306C34076
:101438009396260097020000B38656006780C60080
:101448002307B700A306B7002306B700A305B70014
:101458002305B700A304B7002304B700A303B7000C
:101468002303B700A302B7002302B700A301B70004
:101478002301B700A300B7002300B700678000006E
:1014880093F5F50F93968500B3E5D500939605017E
:10149800B3E5D5006FF0DFF69396270097020000BA
:1014A800B386560093820000E78006FA9380020014
:1014B800938707FF3307F7403306F600E378C3F650
:1014C8006FF0DFF36780000067800000130101FF01
:1014D800232481002322910093040500138505002D
:1014E8002326110023A2010CEFF00F899307F0FFC8
:1014F800630CF5008320C10003248100832441008C
:10150800130101016780000083A7410CE38407FEF3
:101518008320C1000324810023A0F4008324410018
:10152800130101016780000003A7010783278714BF
:10153800638C070403A747001308F001634EE8060D
:101548001318270063060502338307012324C30801
:1015580083A88718130610003316E600B3E8C800FE
:1015680023A417192324D310930620006304D5025B
:101578001307170023A2E700B387070123A4B700C6
:1015880013050000678000009307C7142324F7148D
:101598006FF05FFA83A6C7181307170023A2E700A6
:1015A80033E6C60023A6C718B387070123A4B700EC
:1015B80013050000678000001305F0FF6780000036
:1015C800130101FD2324810103AC0107232E3101FE
:1015D800232C4101232A51012328610123261102CA
:1015E800232481022322910223202103232671012F
:1015F800930A0500138B0500130A10009309F0FFE6
:1016080003298C1463080902832449001384F4FF16
:101618006342040293942400B304990063040B0406
:1016280083A74410638067051304F4FF9384C4FF01
:10163800E31634FF8320C10203248102832441027C
:10164800032901028329C101032A8101832A410157
:10165800032B0101832BC100032C8100130101031B
:10166800678000008327490083A644009387F7FF1B
:10167800638A870423A20400E38806FA832789186B
:1016880033178A00832B4900B377F700639E07005E
:10169800E780060083274900E39477F783278C14B3
:1016A800E38427F96FF0DFF58327C91883A5440879
:1016B8003377F700631C070013850A00E7800600EC
:1016C8006FF05FFD232289006FF01FFB1385050073
:1016D800E78006006FF01FFC130101FE232821019B
:1016E800232C8100232A910023263101138405002D
:1016F800232E110093090500138981C6EFF09FDCA2
:1017080083268900371700009307F7FE83A4460055
:101718003384874093F4C4FF330494001354C40003
:101728001304F4FF1314C400634EE400930500008F
:1017380013850900EFF09FD983278900B3879700A5
:101748006306F50213850900EFF01FD88320C10155
:101758000324810183244101032901018329C10054
:10176800130500001301010267800000B3058040E3
:1017780013850900EFF09FD59307F0FF6304F50484
:1017880083A7C10983268900B384844093E41400A5
:10179800338487401385090023A2960023AE81086D
:1017A800EFF09FD28320C1010324810183244101EA
:1017B800032901018329C100130510001301010247
:1017C800678000009305000013850900EFF01FD023
:1017D800032789009306F000B307E540E3D4F6F643
:1017E80083A6410893E717002322F7003305D54065
:1017F80023AEA1086FF01FF563860512130101FFE0
:1018080023248100232291001384050093040500FA
:1018180023261100EFF01FCB0325C4FF130784FF15
:101828009377E5FF3306F700938581C68326460044
:1018380003A8850093F6C6FF630EC8182322D600B6
:10184800137515003308D6006310050A032384FFB7
:10185800032848003307674083288700138501C79A
:10186800B3876700137818006380A8140323C700A0
:1018780023A66800232413016306081C93E61700B7
:101888002322D7002320F6009306F01F63E8F60A08
:1018980093D73700938617009396360003A8450020
:1018A800B386D50003A5060013D62740930710007A
:1018B800B397C700B3E70701138686FF2326C7003F
:1018C8002324A70023A2F50023A0E6002326E50091
:1018D800032481008320C100138504008324410070
:1018E800130101016FF05FBE032548001375150051
:1018F800631C0502B387D700138501C783268600BA
:1019080093E817003308F700638AA6140326C60075
:1019180023A6C6002324D600232217012320F8007B
:101928006FF09FF66780000093E61700232ED4FE21
:101938002320F6009306F01FE3FCF6F493D69700F5
:1019480013064000636ED60C93D667001385960382
:1019580013868603131535003385A50083260500F5
:10196800130585FF630AD51003A646001376C6FF44
:1019780063F6C70083A68600E318D5FE03A5C60054
:101988002326A7002324D700032481002324E5006D
:101998008320C100138504008324410023A6E600A8
:1019A800130101016FF05FB26318081283258600E6
:1019B8000326C600B387F60093E6170023A6C500E2
:1019C8002324B6002322D7003307F7002320F7008B
:1019D8006FF01FF013751500B387D7006310050269
:1019E800032584FF3307A7408326C7000326870003
:1019F800B387A7002326D60023A4C60013E6170042
:101A080083A681082322C70023A4E500E3E2D7ECDC
:101A180083A5410913850400EFF01FCC6FF05FEB3D
:101A2800130640016374D602130640056364D606A4
:101A380093D6C7001385F6061386E60613153500F8
:101A48006FF09FF1B387D7006FF05FEB1385C60582
:101A58001386B605131535006FF01FF023AAE500AD
:101A680023A8E5002326A7002324A7002322170183
:101A78002320F8006FF0DFE503A845001356264041
:101A8800930710003396C7003366060123A2C500EA
:101A98006FF01FEF13064015636CD60093D6F7005E
:101AA8001385860713867607131535006FF0DFEA6E
:101AB80013064055636CD60093D627011385D607C5
:101AC8001386C607131535006FF01FE91305803F0D
:101AD8001306E0076FF05FE893E617002322D700AC
:081AE8002320F6006FF0DFDEA1
:101AF0003000000031000000320000003300000020
:101B000034000000350000003600000037000000FF
:101B10003800000039000000610000006200000091
:101B20006300000064000000650000006600000023
:101B300048656C6C6F2066726F6D205F69736174AD
:101B400074790A004552524F523A205F6B696C6CAF
:101B5000206E6F742079657420696D706C656D6599
:101B60006E7465640A0000004552524F523A205F7D
:101B7000756E6C696E6B206E6F7420796574206968
:101B80006D706C656D656E7465640A004552524FE8
:101B9000523A205F67657474696D656F6664617938
:101BA000206E6F742079657420696D706C656D6549
:101BB0006E7465640A0000004552524F523A205F2D
:101BC0006C696E6B206E6F742079657420696D701E
:101BD0006C656D656E7465640A000000300000007D
:101BE000310000003200000033000000340000002B
:101BF000350000003600000037000000380000000B
:101C00003900000061000000620000006300000075
:0E1C10006400000065000000660000000A008D
:042000004800008014
:10200800DC1B0080E01B0080E41B0080E81B0080D4
:10201800EC1B0080F01B0080F41B0080F81B008084
:10202800FC1B0080001C0080041C0080081C008031
:102038000C1C0080101C0080141C0080181C0080E0
:1020480000000000342300809C23008004240080CA
:102058000000000000000000000000000000000078
:102068000000000000000000000000000000000068
:102078000000000000000000000000000000000058
:102088000000000000000000000000000000000048
:102098000000000000000000000000000000000038
:1020A8000000000000000000000000000000000028
:1020B8000000000000000000000000000000000018
:1020C8000000000000000000000000000000000008
:1020D80000000000000000000000000000000000F8
:1020E80000000000000000000100000000000000E7
:1020F8000E33CDAB34126DE6ECDE05000B000000AC
:1021080000000000000000000000000000000000C7
:1021180000000000000000000000000000000000B7
:1021280000000000000000000000000000000000A7
:102138000000000000000000000000000000000097
:1024780070240080702400807824008078240080F4
:1024880080240080802400808824008088240080A4
:102498009024008090240080982400809824008054
:1024A800A0240080A0240080A8240080A824008004
:1024B800B0240080B0240080B8240080B8240080B4
:1024C800C0240080C0240080C8240080C824008064
:1024D800D0240080D0240080D8240080D824008014
:1024E800E0240080E0240080E8240080E8240080C4
:1024F800F0240080F0240080F8240080F824008074
:10250800002500800025008008250080082500801F
:1025180010250080102500801825008018250080CF
:10252800202500802025008028250080282500807F
:10253800302500803025008038250080382500802F
:1025480040250080402500804825008048250080DF
:10255800502500805025008058250080582500808F
:10256800602500806025008068250080682500803F
:1025780070250080702500807825008078250080EF
:10258800802500808025008088250080882500809F
:10259800902500809025008098250080982500804F
:1025A800A0250080A0250080A8250080A8250080FF
:1025B800B0250080B0250080B8250080B8250080AF
:1025C800C0250080C0250080C8250080C82500805F
:1025D800D0250080D0250080D8250080D82500800F
:1025E800E0250080E0250080E8250080E8250080BF
:1025F800F0250080F0250080F8250080F82500806F
:10260800002600800026008008260080082600801A
:1026180010260080102600801826008018260080CA
:10262800202600802026008028260080282600807A
:10263800302600803026008038260080382600802A
:1026480040260080402600804826008048260080DA
:10265800502600805026008058260080582600808A
:10266800602600806026008068260080682600803A
:1026780070260080702600807826008078260080EA
:10268800802600808026008088260080882600809A
:10269800902600809026008098260080982600804A
:1026A800A0260080A0260080A8260080A8260080FA
:1026B800B0260080B0260080B8260080B8260080AA
:1026C800C0260080C0260080C8260080C82600805A
:1026D800D0260080D0260080D8260080D82600800A
:1026E800E0260080E0260080E8260080E8260080BA
:1026F800F0260080F0260080F8260080F82600806A
:102708000027008000270080082700800827008015
:1027180010270080102700801827008018270080C5
:102728002027008020270080282700802827008075
:102738003027008030270080382700803827008025
:1027480040270080402700804827008048270080D5
:102758005027008050270080582700805827008085
:102768006027008060270080682700806827008035
:1027780070270080702700807827008078270080E5
:102788008027008080270080882700808827008095
:102798009027008090270080982700809827008045
:1027A800A0270080A0270080A8270080A8270080F5
:1027B800B0270080B0270080B8270080B8270080A5
:1027C800C0270080C0270080C8270080C827008055
:1027D800D0270080D0270080D8270080D827008005
:1027E800E0270080E0270080E8270080E8270080B5
:1027F800F0270080F0270080F8270080F827008065
:102808000028008000280080082800800828008010
:1028180010280080102800801828008018280080C0
:102828002028008020280080282800802828008070
:102838003028008030280080382800803828008020
:1028480040280080402800804828008048280080D0
:102858005028008050280080582800805828008080
:102868006028008060280080682800806828008030
:1028780048200080000000700000001000000020C8
:0C28880048200080FFFFFFFF000002005E
:040000058000000077
:00000001FF
